:1000000012C0189518951895189518951895189563
:100010001895189518950ECC18951895189518954B
:100020001895189518958FE58DBFC0E4E8E34E2E1E
:1000300084E08EBFD4E0F4E05F2EEEEFF3E0A0E6C4
:10004000B0E084B7082E877F84BF8FE181BD80E058
:1000500081BD88278D933197E9F783E289B980E0E4
:1000600080BD88E18AB96624B89A8E9AA09AA39A2C
:10007000A19A579A78948BB78F7B8BBF8F9A979A58
:1000800082E08093750180E080937C0181E0809321
:100090007A0180E080937B0180E08093760131D902
:1000A00080ED97E01DDAC098969883E289B980E0E8
:1000B00080BDB998ADE9B1E0ECEAFBE120DA8DE072
:1000C000ADE9B1E08F9371D98F918D9388278C938F
:1000D000ADE9B1E06AD9E8EBFBE111DA8DE0ADE919
:1000E000B1E08F9362D98F918D9388278C93ADE97E
:1000F000B1E05BD9E2ECFBE102DA8DE0ADE9B1E021
:100100008F9353D98F918D9388278C93ADE9B1E06C
:100110004CD9ECECFBE1F3D98DE0ADE9B1E08F9384
:1001200044D98F918D9388278C93ADE9B1E03DD967
:10013000E8EDFBE1E4D97FD280ED97E0D1D915D984
:1001400071D3FDCFA5E6B1E011968C91A1E6B1E0A7
:100150008C93A5E6B1E08C91A2E6B1E08C93D3DC60
:1001600010EAE8DCA1E6B1E01C91E4DCA2E6B1E033
:100170001C91E0DCA881B9811C91DCDCD2DC8AE036
:1001800090E0AED90895A5E6B1E011968C91A1E674
:10019000B1E08C93A5E6B1E08C91A2E6B1E08C933E
:1001A000B2DC10EAC7DCA1E6B1E01C91C3DCA2E638
:1001B000B1E01C91BFDCA7DC11EABCDCD8DCA88173
:1001C000B9811C93AEDC0895969AA89AC09A50D82B
:1001D000E4EEFBE120D925D900917601003009F049
:1001E00004C0A0EDB2E05AD953D942D8E4EEFBE105
:1001F00012D917D900917601003009F004C0A0EDA2
:10020000B2E04CD945D934D8E4EEFBE104D909D9A0
:1002100000917601003009F004C0A0EDB2E03ED9B3
:1002200037D926D8E4EEFBE1F6D8FBD80091760169
:10023000003009F004C0A0EDB2E030D929D918D8B7
:10024000E4EEFBE1E8D8EDD800917601003009F04A
:1002500004C0A0EDB2E022D91BD90AD8E4EEFBE13C
:10026000DAD8DFD800917601003009F004C0A0EDA3
:10027000B2E014D90DD9FCD7E4EEFBE1CCD8D1D84B
:1002800000917601003009F004C0A0EDB2E006D97B
:10029000FFD884EF91E024D900917B01003009F070
:1002A00004C0E8EEFBE1B7D8BCD800917B01013077
:1002B00009F035C0EAEFFBE1AED8B3D8D9D7E4EE08
:1002C000FBE1A9D8AED800917601003009F004C056
:1002D000A0EDB2E0E3D8DCD8CBD7E4EEFBE19BD8CD
:1002E000A0D800917601003009F004C0A0EDB2E082
:1002F000D5D8CED8BDD7E4EEFBE18DD892D8009109
:100300007601003009F004C0A0EDB2E0C7D8C0D833
:1003100084EF91E0E5D8EAE0FCE17DD882D8A8D767
:10032000E4EEFBE178D87DD800917601003009F049
:1003300004C0A0EDB2E0B2D8ABD89AD7E4EEFBE1AE
:100340006AD86FD800917601003009F004C0A0EDA2
:10035000B2E0A4D89DD88CD7E4EEFBE15CD861D89C
:1003600000917601003009F004C0A0EDB2E096D80B
:100370008FD880ED97E0B4D800917C01003009F06F
:1003800004C0ECE1FCE147D84CD800917C0101307D
:1003900009F004C0EEE2FCE13ED843D869D70091F1
:1003A0007601003009F004C0A0EDB2E077D870D833
:1003B000E4EEFBE130D835D800917601003009F049
:1003C00004C0E0E4FCE15CD863D888EE93E088D810
:1003D000E4EEFBE120D825D885E089B980E080BD36
:1003E00080ED97E07DD8ECE5FCE115D81AD880EDDA
:1003F00097E076D8ECE5FCE10ED813D800917601B1
:10040000003009F004C0E4E6FCE13AD841D8AFE698
:10041000B1E00ADA80E08093790100917A0100303E
:1004200009F010C0E2E8FCE12BD832D80091750148
:10043000013009F002C08FEF13D80091750102302E
:1004400009F000C040E45DE063E070E0AFE6B1E0D9
:100450000D911D912D913C9121DA0CF401C069C0E0
:10046000ABD7ABE6B1E08C9300916B01013009F0A2
:1004700057C0A2D7ABE6B1E08C9300916B0101307D
:1004800009F04DC0C09AA3D7AAE6B1E08C930091C1
:100490006A010F3F09F003C081E080937901009168
:1004A0007901013009F038C080916A0180936401BC
:1004B00000917A01003009F018C0009175010130F7
:1004C00009F004C0A4E6B1E08C91CAD7009175018F
:1004D000023009F009C0A0E2B4E0E4E6F1E04ADA53
:1004E000DBD7E8E8FCE1CCD717C05A924A92A5E6E0
:1004F000B1E08D919C91A42DB52D8D939C9382E0BC
:100500003AD7E4E6F1E0FA93EA931CDE249682E01F
:100510002ED7A5E6B1E042D7AFE6B1E085D9A4CFAA
:10052000C09885B391E0892785BBAFE6B1E027D7B6
:1005300089CF00917A01003009F004C0EAE8FCE1BB
:100540009FD7A6D700917A01013009F055C0E2E8A3
:10055000FCE196D79DD7A5E6B1E08D919C91A7E6E9
:10056000B1E08D939C9380E190E0A5E6B1E08D939E
:100570009C93A7E6B1E04D915C91A5E6B1E00D91A9
:100580001C910417150708F033C05A924A92A5E649
:10059000B1E08D919C91A42DB52D8D939C9382E01B
:1005A000EAD6E3E6F1E0FA93EA93EDDD249682E001
:1005B000DED680916301809369010091750101305D
:1005C00009F004C0A9E6B1E08C914AD70091750109
:1005D000023009F009C0A0E2B4E0E9E6F1E0CAD9CE
:1005E0005BD7E8E8FCE14CD7A5E6B1E0D7D6C1CFB0
:1005F000EAE8FCE145D74CD7C09A0091760100307B
:1006000009F004C0E0E9FCE13BD742D7A89800918B
:100610007601003009F004C0EAEAFCE131D738D7AE
:10062000969800917601003009F004C0E2ECFCE1FC
:1006300027D72ED70895E8EDFCE122D729D7E2E0AD
:10064000F0E0F6D6ADE9B1E0F5D9A2E3B3E08C93E2
:10065000009132034EE0040FA8E3B3E00C93ECEDFD
:10066000FCE10ED7A0E2B4E0E8E3F3E039D914D717
:10067000E6EEFCE105D70CD784E690E031D7A2E0A6
:10068000B2E0EAEEFCE13BD7A8E3B3E08C91825004
:100690008C93AFE2B3E0E8E3F3E06CD9EFE2F3E090
:1006A000A2E0B2E082D681D9A2E0B2E07ED6EEEE40
:1006B000FCE125D781E080933103ABECB2E0E2E3CB
:1006C000F3E058D9EBECF2E0A2E0B2E06ED66DD9DF
:1006D000A9E2B3E0E4E0FDE112D7E9E2F3E0A2E051
:1006E000B2E063D662D9409132030091310304171E
:1006F00010F009F020C080913103EDE9F1E001E054
:100700000A93A9E2B3E05CD9A9E2B3E08C91A7E334
:10071000B3E08C93ACE2B3E0E7E3F3E02BD9ECE297
:10072000F3E0A2E0B2E041D640D9A1E3B3E08C917E
:100730008F5F8C93D8CFA2E0B2E0B0D68AE190D69A
:100740000895A9E1B3E0E8E0FDE1D9D6A4E0B3E083
:10075000EEE0FDE1D4D6E0E1FDE192D699D684EF5A
:1007600091E0BED6E4E1FDE18BD6A9E1B3E096D6F7
:10077000EAE1FDE185D68CD6E2E3F0E059D6ECE182
:10078000FDE17ED682E26CD6A4E0B3E087D682E2B9
:1007900067D67ED6EEE1F0E04BD6E0E1FDE170D623
:1007A00077D688EE93E09CD6ECE1FDE169D682E253
:1007B00057D6AFEEB2E072D682E252D669D6EDE2FB
:1007C000F0E036D6A4E0B3E0E6E2FDE198D6ECE155
:1007D000FDE156D682E244D6A4E0B3E05FD682E2E1
:1007E0003FD656D6EAE0F0E023D6E0E1FDE148D678
:1007F0004FD688EE93E074D6E8E2FDE141D6089545
:10080000E8EDFCE13DD644D684EF91E069D6E4E121
:10081000FDE136D6A9E1B3E041D63AD6EEE1F0E00B
:1008200007D60895E8EDFCE12BD632D681E080931F
:100830003A0380E080933B0300913B03003009F0D2
:10084000A7C280E080936A01AEE7B1E0EBD70091E8
:100850006A010D3081E008F080E08F9300916A0119
:100860000D3080E010F009F081E09F91892B882302
:1008700009F41EC022D6AAE6B1E08C9300916A0169
:10088000013010F009F001C012C000916A010E3170
:1008900010F009F001C00BC0AAE6B1E08C91AEE700
:1008A000B1E08F9382D58F918D9388278C93CFCF92
:1008B000AEE7B1E0EEE2FDE1C3D809F00BC0E0E441
:1008C000FDE1DED5E5D5E2E4FDE1DAD5E1D581E073
:1008D00080933B03AEE7B1E0E8E5FDE1B1D809F074
:1008E00007C0EEE5FDE1CCD5D3D581E080933B0395
:1008F000AEE7B1E0E2E6FDE1A3D809F019C0E8E611
:10090000FDE1BED5C5D5A89881E080933B03C09892
:100910009698A89883E289B980E080BDAEE5B1E001
:10092000B4D780E190E0A5E6B1E08D939C934CDCD8
:10093000AEE7B1E0E0E8FDE183D881E009F080E0D6
:100940008F93AEE7B1E0E8E8FDE17AD881E009F005
:1009500080E09F91892B8F93AEE7B1E0E0E9FDE164
:100960006FD881E009F080E09F91892B882309F4FA
:100970004FC1E6E9FDE184D5AFEEB2E053D780E0A8
:1009800080936A01AFE6B1E04FD700916A010D3064
:1009900081E008F080E08F9300916A010D3080E0E3
:1009A00010F009F081E09F91892B882309F44DC054
:1009B00084D5AAE6B1E08C9300916A01013010F071
:1009C00009F001C02CC000916A01013010F009F05B
:1009D00001C025C000916A010D3081E008F080E07F
:1009E0008F9300916A010D3080E010F009F081E0F2
:1009F0009F91892B882309F40FC0AAE6B1E08C915E
:100A00002FD5AAE6B1E08C91AFEEB2E08F93CDD4B2
:100A10008F918D9388278C93AFE6B1E005D7AFE631
:100A2000B1E0ADD440E854E86EE170E0AFE6B1E08B
:100A30000D911D912D913C9131D714F009F001C019
:100A400003C08DE080936A01A0CFE0E4FDE118D5FA
:100A50001FD5E2EAFDE114D5EFEEF2E0A9E1B3E043
:100A6000A4D7AFEEB2E01AD513D5E6EBFDE108D579
:100A70000FD5E3E0F0E0DCD484EF91E031D58BE2F8
:100A8000EFD48BE2EDD48BE2EBD4E2E0F0E0D0D413
:100A9000E8EDFCE1F5D4FCD4E2E0F0E0C9D4E8E212
:100AA000FDE1EED4F5D4E1E0F0E0C2D4E8E2FDE10E
:100AB000E7D4EED4E4E0F0E0BBD4AEE7B1E0E8E8A0
:100AC000FDE1BED709F008C03CDEE8EDFCE1D8D47A
:100AD000DFD4E2E0F0E0ACD4AEE7B1E0E0E9FDE184
:100AE000AFD709F001C08CDEAEE7B1E0E0E8FDE190
:100AF000A7D709F08AC0E6EDFDE1C2D4C9D4ADE9BB
:100B0000B1E090D680E080936A01AFE6B1E08CD688
:100B100000916A010F3681E008F080E08F93009128
:100B20006A010F3680E010F009F081E09F91892B77
:100B3000882309F433C0C1D4AAE6B1E08C930091B4
:100B40006A01013010F009F001C012C000916A0181
:100B50000E3110F009F001C00BC0AAE6B1E08C9193
:100B6000ADE9B1E08F9321D48F918D9388278C9339
:100B7000AFE6B1E004D440E854E86EE170E0AFE6DF
:100B8000B1E00D911D912D913C9188D614F009F0A2
:100B900001C003C08FE680936A01BACFA89A40E8EB
:100BA00054E86EE170E0AFE6B1E00D911D912D913A
:100BB0003C9174D60CF401C01EC0E0E0F0E0ADE959
:100BC000B1E07BE712D7A9E1B3E034D7A9E3B3E002
:100BD0008C9300913903023010F009F001C001C07C
:100BE000D8D0ADE9B1E0E0EEFDE189D424DD80EDBF
:100BF00097E076D409C0ADE9B1E0EEEEFDE17FD437
:100C00001ADD80ED97E06CD4A89881E080933B03D7
:100C1000AEE7B1E0E2E0FEE113D709F00EC0E0E09C
:100C2000F0E0ADE9B1E094E6EBD6EAE0FEE128D4ED
:100C30002FD4ADE9B1E032D42BD4AEE7B1E0E8E196
:100C4000FEE1FED609F00AC0EEE1FEE119D420D49F
:100C500080E080937C0181E080933B03AEE7B1E0CC
:100C6000EAE3FEE1EDD609F00AC0E0E4FEE108D4D3
:100C70000FD481E080937C0181E080933B03AEE759
:100C8000B1E0E8E5FEE1DCD609F00AC0EEE5FEE100
:100C9000F7D3FED380E080937A0181E080933B0319
:100CA000AEE7B1E0EEE7FEE1CBD609F00AC0E4E83A
:100CB000FEE1E6D3EDD381E080937A0181E0809379
:100CC0003B03AEE7B1E0ECE9FEE1BAD609F00AC0B9
:100CD000E2EAFEE1D5D3DCD381E080937B0181E0C1
:100CE00080933B03AEE7B1E0E6EBFEE1A9D609F065
:100CF0000AC0ECEBFEE1C4D3CBD380E080937B0150
:100D000081E080933B03AEE7B1E0E0EDFEE198D6F1
:100D100009F00AC0E6EDFEE1B3D3BAD382E08093D6
:100D2000750181E080933B03AEE7B1E0EAEEFEE1BE
:100D300087D609F00AC0E0EFFEE1A2D3A9D381E093
:100D40008093750181E080933B03AEE7B1E0E4E07E
:100D5000FFE176D609F00AC0EAE0FFE191D398D32B
:100D600080E08093760181E080933B03AEE7B1E0C1
:100D7000E6E2FFE165D609F00AC0ECE2FFE180D3CC
:100D800087D381E08093760181E080933B0354CD4B
:100D9000089580E080934403A2E0B2E0E8E4FFE13C
:100DA000AED3A9E1B3E046D6A7E3B3E08C9380913C
:100DB000370380933203ABECB2E0E7E3F3E0DAD53C
:100DC000EBECF2E0A2E0B2E0F0D2EFD5A2E0B2E0CC
:100DD000ECD2E0E5FFE193D381E08093310382E040
:100DE00090E0A5E4B3E08D939C93AEECB2E01AD50D
:100DF000ACE2B3E017D54091320300913103041700
:100E000010F009F08AC080913103E9E1F3E001E0DC
:100E10000A93AEECB2E0D4D580914503E9E1F3E06A
:100E200001E00A93ACE2B3E0CBD5409132030091EC
:100E30003103041709F04EC000913203023081E003
:100E400009F080E08F9300913203043081E009F0D3
:100E500080E09F91892B8F9300913203063081E0CF
:100E600009F080E09F91892B8F9300913203083025
:100E700081E009F080E09F91892B8F9300913203EC
:100E80000A3081E009F080E09F91892B8F930091D7
:100E900032030C3081E009F080E09F91892B8F9321
:100EA000009132030E3081E009F080E09F91892BA0
:100EB000882309F40AC080914503E9E1F3E001E0E9
:100EC0000A93ACE2B3E07CD505C0ACE2B3E0E4E564
:100ED000FFE115D3ECE2F3E0A2E0B2E066D265D523
:100EE000EEECF2E0A2E0B2E060D25FD5AEECB2E0B0
:100EF00099D4ACE2B3E096D4A1E3B3E08C918F5FD8
:100F00008C93A1E3B3E08C918F5F8C93A5E4B3E065
:100F100045D2A5E4B3E042D26ECFA2E0B2E045D222
:100F2000E6E5FFE1ECD281E08093310382E090E0DE
:100F3000A5E4B3E08D939C93ADE9B1E07BD5A7E345
:100F4000B3E08C938091370380933203ABECB2E033
:100F5000E7E3F3E00FD5EBECF2E0A2E0B2E025D25C
:100F600024D5A2E0B2E066D5A9E4B3E08D9388274A
:100F70008C934091320300913103041710F009F073
:100F80006EC080913103EDE9F1E001E00A93AEEC2F
:100F9000B2E016D5AEECB2E08C91AEE3B3E08C9348
:100FA00080914503EDE9F1E001E00A93ACE2B3E0A2
:100FB00007D5ACE2B3E08C91AFE3B3E08C93009142
:100FC000310341E0041BA8E4B3E00C930091480313
:100FD00048E020D5A7E4B3E08C93A7E4B3E09C916C
:100FE000AEE3B3E099D207E040914703041BA7E4C6
:100FF000B3E00C93A7E4B3E09C91AFE3B3E084D2F9
:1010000000913E0340913F03040FAEE3B3E00C9325
:10101000ABECB2E0EEE3F3E0ADD4EBECF2E0A2E057
:10102000B2E0C3D1C2D4A9E4B3E0B8D1A9E4B3E03B
:10103000B5D1A1E3B3E08C918F5F8C93A5E4B3E0CD
:10104000ADD100914703013009F008C0A5E4B3E039
:10105000A5D1A1E3B3E08C918F5F8C938ACF80916F
:10106000490380933203E8EAFBE1BDD3E2E3F3E016
:10107000D080EE24FF240027B9D204D3EDE0F0E0C5
:10108000A3E3B3E097D4E3E3F3E02FD5EDE0F0E0A2
:101090004BD2A7E3B3E0DC920091370341E0041B9D
:1010A000A2E3B3E00C9380914B03806880934B03E1
:1010B00080914B038F7B80934B03ABE4B3E08C9127
:1010C00087FB0EF0D4C0E8EDFCE1DAD1E1D1E2E03B
:1010D000F0E0AED1EEE5FFE1D3D1A0E2B4E0E2E38F
:1010E000F3E0FED3D9D1D4D185E090E0F9D1ABE4DF
:1010F000B3E08C9186FB0EF41BC080E080936A0104
:1011000000916A010D3081E008F080E08F9300913A
:101110006A010D3080E010F009F081E09F91892B89
:10112000882309F405C0C9D1AAE6B1E08C93E8CFC1
:1011300082E390E0D5D1A2E0B2E0B0D18AE190D1D3
:10114000ADE9B1E06FD380E08093370300913703BE
:101150000A3081E008F080E08F93009137030A3075
:1011600080E010F009F081E09F91892B882309F439
:1011700010C0A3D1A7E3B3E08C93A7E3B3E08C91B5
:10118000ADE9B1E08F9311D18F918D9388278C9326
:10119000DDCFADE9B1E046D380E080933703009125
:1011A00037030A3081E008F080E08F930091370325
:1011B0000A3080E010F009F081E09F91892B8823AC
:1011C00009F410C07AD1A7E3B3E08C93A7E3B3E0AE
:1011D0008C91ADE9B1E08F93E8D08F918D93882702
:1011E0008C93DDCF81E0EDE9F1E002E00A93ACE21F
:1011F000B3E0E6D3ACE2B3E0E8E6FFE121D409F0E6
:1012000006C080914B038F7780934B030EC0ECE6B2
:10121000FFE136D13DD180914B03806880934B0331
:1012200080914B038F7B80934B03E5E0F0E000D18E
:10123000A89884EF91E054D1A89A84EF91E050D11E
:10124000A89884EF91E04CD1A89AA4E4B3E08C91E3
:101250008F5F8C9300914403043110F009F001C0BA
:1012600005C080914B038F7780934B0326CF089561
:10127000A0EDB2E0D7D280E080936A01AFE6B1E0A2
:10128000D3D200916A010D3081E008F080E08F93A5
:1012900000916A010D3080E010F009F081E09F912B
:1012A000892B882309F42CC08DD0AAE6B1E08C9359
:1012B00000916A010D3010F009F001C00BC0AAE6E0
:1012C000B1E08C91A0EDB2E08F936FD08F918D93B0
:1012D00088278C93AFE6B1E052D040EC56EC6DE23B
:1012E00070E0AFE6B1E00D911D912D913C91D6D209
:1012F00014F009F001C003C08DE080936A01C1CFF2
:101300000895E4E0F0E094D0AB98E4E0F0E090D011
:10131000AB9AE2E0F0E08CD0A99AE1E0F0E088D06E
:10132000A998E1E0F0E084D0A99AE1E0F0E080D073
:10133000A998E1E0F0E07CD0AB9884EF91E0D0D0C8
:10134000AB9A84EF91E0CCD0AB9884EF91E0C8D019
:10135000AB9A84EF91E0C4D0AB9884EF91E0C0D019
:10136000AB9A84EF91E0BCD0089500000895481A2C
:101370008827580A0895480E8827581E08950D9109
:101380001D912D913C9181E0080F8827181F281F7F
:10139000381F3C932E931E930E930895ED91FC916C
:1013A000EF5FFF4FFC93EE9308958F938D91882309
:1013B000E9F711978F91089580916001882309F0D2
:1013C00081E0089580916001882309F408950F92C7
:1013D0009F93AF93BF937F93809160018823E1F344
:1013E000F894809160018A958093600190915E01EC
:1013F000A0E6B0E0A90F0024B01D8C9193959E3F0C
:1014000009F4992790935E0178947F91BF91AF91F1
:101410009F910F900895E3D1802D11F005D0FBCF5F
:1014200008958DE001D08AE05D9BFECF8CB90895D0
:1014300088EE93E055D03197D9F708953197F1F7B9
:101440000895689462F80895E89462F808958F9377
:101450009F938BE890E00197F1F79F918F9108950A
:1014600080952AE090E0089410F4979802C0979A2B
:101470000000EDDFECDF969587952A95A9F7089592
:10148000C895802D882319F0EBDF3196F9CF0895A8
:101490008DE0E6DF8AE0E4CFA0E2B4E08D9188231E
:1014A00011F0DEDFFBCF08958F939F938BE890E0E0
:1014B0000197F1F79F918F910895B19B02C0882702
:1014C000089529E0B199FECFEFDFEEDFEDDF8894DC
:1014D000B19908942A9519F087959795F6CF0895B4
:1014E000EF93FF93EE27E82BE92B31F0EDECFAE0D8
:1014F0003197F1F70197D1F7FF91EF9108956FD1EF
:101500000D920020E1F70895903029F08C91880F1A
:101510009A95E9F78C930895903029F08C918695EF
:101520009A95E9F78C9308953DD0992711278F2D2F
:10153000880F80E8F82A802F881F08F41FEF41F0F9
:101540008F57082F07FD04C0003240F08FEF01C015
:101550008827982FD82EE82EF82E09C08FE1801BFF
:10156000082FF694E794D79497950A95D1F711230D
:1015700051F09095D094E094F09481E0980F8827F2
:10158000D81EE81EF81E0F2DFE2CED2CD92E089526
:10159000D094E094F09491E0D90E9927E91EF91EB9
:1015A00010950895D190E190F190019108952191C5
:1015B0003191419151910895102F90E8FF0C001F37
:1015C0000927990FF7941078652F90E8440F551F5D
:1015D0005927990F4795607800380895FF0C90E8D7
:1015E0009027110F9795F794092F0895102FBD2C70
:1015F000DE2CEF2CF02E11234AF4B094D094E0941A
:10160000F0949FEFB91AD90AE90AF90A0EE1FF200E
:1016100039F4FE2CED2CDB2CBB240850C2F766C03D
:1016200032F00A95BB0CDD1CEE1CFF1CF9CF01D07B
:10163000D5CFB7FE089590E8B91611F4D0FE0895FD
:101640009FEFD91AE90AF90A09F403950895502F72
:101650002D2D3E2D4F2D612F08952DEC3CEC4CECA3
:101660005DE366270FC09EDFF2DFDD24EE2490E805
:10167000F92E0FE307C09BDF05C02227332740E286
:1016800051E46627552351F1002381F195DF71F173
:101690001627005850580894050B18F407FD03C08E
:1016A00025C007FD23C0469537952795F694E79406
:1016B000D79422D0FF202AF0DD0CEE1CFF1C015035
:1016C00073F09D2D969548F0DD203AF4EE202AF433
:1016D00091E0D90E9927E91EF91E80CF07C09FE738
:1016E000092FF92A9FEFD92EE92E0895DD24EE2443
:1016F000FF240027112708959F929924AA24BB2430
:1017000088E1D216E306F40628F0D21AE30AF40AB6
:10171000089401C08894991CAA1CBB1CDD0CEE1C0B
:10172000FF1C8A9571F7D92CEA2CFB2C9F90089509
:101730000AF045D053CF5FE322273327442701C067
:1017400036DF3ADF5038B1F3003899F3902F951B0C
:101750008BF312F434D0FACF983118F022273327C4
:101760004427983028F0232F342F44279850F9CF5E
:10177000992329F04695379527959A95D9F7912F72
:10178000962742F014D0B0F6F794E794D7940F5F01
:101790008BF6A5CF10D051F008F4FADEFF2052F2FC
:1017A000DD0CEE1CFF1C0150CBF799CF9FCFD20E62
:1017B000E31EF41E0895D21AE30AF40A0895DF9294
:1017C000EF92FF920F931F93D22EE32EF42E052F4C
:1017D000162F6F915F914F913F912F910895C8956A
:1017E000319600200895FBDF202DF9DF302DF7DF43
:1017F000402DF5DF502D089507FB00680EF40F779C
:1018000057FB50680EF45F7707FD02C057FF05C015
:10181000D216E306F406050708952D153E054F057B
:101820005007089582E001C084E099279D938A952E
:10183000E9F708957F930F93AF93BF938F939F938F
:101840008FB78F93809160010EEF081B19F49CB144
:10185000F8DD12C000915F01A0E6B0E077279CB1EF
:10186000A00FB71F9C9383958093600103950E3F53
:1018700009F4002700935F018F918FBF9F918F9193
:10188000BF91AF910F917F9118956FB7F89488270A
:1018900093E08D939A95E9F76FBF089504171507A4
:1018A000260737070895000F111F221F331F0895C1
:1018B00000951095209530950F5F1F4F2F4F3F4F8C
:1018C0000895019110810EC00191119121913081F3
:1018D0000BC00191108117FF05C03FEF2FEF04C02F
:1018E000008111272227332737FF03C0E1DF8DE274
:1018F0008D93CF93DF93CF92DF92EF92AA24BB24F4
:10190000CC24DD24EE2440E2CAE0DD2755E093E359
:101910008881890F87FD9F7083FD907F891B899344
:101920005A95A9F7C0DFAA1CBB1CCC1CDD1CEE1C01
:101930004A9551F7E894EFE0FF2782910ED0EB3003
:10194000E0F71EF068948A2D0CD088278D93EF90D5
:10195000DF90CF90DF91CF910895982F829501D09D
:10196000892F8F70805D26F0803309F40895689484
:101970008D93089541E003C042E001C044E0E40FCC
:101980008827F81F8291982F829505D0892F03D040
:101990004A95C1F707C08F708A3008F0895F805D73
:1019A0008D93089588278D93089581918D93882331
:1019B000E1F7089594E081918D939A95E1F7089568
:1019C00009919191992351F08A95D9F73197819195
:1019D0008D930A9519F08823D1F70895E3CFE19903
:1019E000FECFEEBBFFBB31960895F9DF8D917B37BB
:1019F00029F48DBBE29AE19A8823B9F777270895F5
:101A0000EEDFE09A8DB38D93882319F09A95C1F794
:101A10009D930895FF93881BF9E0001FFA9511F438
:101A2000FF910895881F841B18F4840F8894F5CFC4
:101A30000894F3CF8FEF83959D919923E1F7089553
:101A4000689401C0E894AF93BF938D9116F0919183
:101A500002C0C5DE902D891718F011F48823A9F76C
:101A6000BF91AF9108959EDD80E003C09BDD802F84
:101A70008078882321F0DF92EF92FF920F938F936B
:101A80009BDD802F839512F431DE1BC080958A95F3
:101A9000885E0AF415C088501AF40CD0D92210C000
:101AA000DD2488501AF406D0E9220AC0EE2402D0C0
:101AB000F92206C09FEF8770990F8A95EAF708957B
:101AC0008DDD8F918823D9F35F914F913F912F91B5
:101AD0000F9392DE0F9199F390F302D0506831CEBC
:101AE0005FE340E83327222708955CDD0F930F77EB
:101AF00022DEBDDF8F918078082B0895AC98AD98D9
:101B0000A498A5980895A59AA49803D0A59801D063
:101B1000A49AEF93FF93EAE0F0E090DCFF91EF915D
:101B20000895A59AA49AF5DFA5989D9BFECFF1DFB5
:101B3000A498EFCF0894111F01C0110F69F0A59A66
:101B400018F40000A49802C0A49A00C0E2DFA5988F
:101B50009D9BFECFDEDFF1CFA59AA498DADFA59892
:101B60009D9BFECFE8949C99689462F8D2CF08942C
:101B700001C08894331F11E0A59AA498CADFA598E4
:101B80009D9BFECFC6DF88949C990894111FA0F7F7
:101B9000A59A379510F4A49801C0A49ABADFA59825
:101BA0009D9BFECFB6DF089500000040566572731E
:101BB000696F6E20312E310050726F6772616D6DEA
:101BC0000000676573746172746574002D2D2D2D8E
:101BD0002D2D2D2D2D2D00002043534420616B749D
:101BE000697620004F4B00005E534143443A203158
:101BF000372C30342C322C3100005E534143443AB0
:101C00002031372C30332C3200005E534143443AAC
:101C10002031372C30342C322C3200005E534143BB
:101C2000443A2031372C30312C322C3100005E53B5
:101C30004143443A2031372C30312C322C320000D1
:101C40005765636873656C652064696520446174D9
:101C5000656E72617465202E2E2E0000434F4E4E2D
:101C600045435400426567696E6E65206D69742056
:101C7000446174656E61757367616265202E2E2EF6
:101C8000000043414D5F4200200043414D5F45004D
:101C9000446174656E2077757264656E2075656247
:101CA000657274726167656E00004B616D6572618B
:101CB000207769726420616267657374656C6C7407
:101CC00000004175666E61686D656D6F64757320A7
:101CD0006265656E646574004154000041545E5352
:101CE00053544B3D00002C3000004430000038318C
:101CF00030333031323138303832303238313032BE
:101D000038440000303400003131353500003400F3
:101D1000617400006174642000003B006174202B3A
:101D20007674733D00003100617420686E00434F8B
:101D30004E4E45435420393630302F524C5000001F
:101D4000000056657262696E64756E672065746125
:101D5000626C696572742E0052494E47000041540E
:101D6000410042494C44000042696C646D6F6475E7
:101D70007320776972642067656C6164656E00002A
:101D8000434F4E534D530000434F4E4C41440000CF
:101D9000525545434B0045696E676162653F3A2085
:101DA00000004469652045696E67616265206C6169
:101DB000757465743A004265656E64652064696592
:101DC00020446174656E76657262696E64756E67D3
:101DD000202E2E2E00006174642A313030233B0007
:101DE000534D532076657273656E64657400534D70
:101DF00053206E696368742076657273656E6465DE
:101E0000740047555443484B00004775746861623D
:101E1000656E202E2E2E0000434F4E524C0047651B
:101E200072696E6765204175666C6F6573756E6764
:101E30002067657365747A740000434F4E52480002
:101E4000486F6865204175666C6F6573756E6720B5
:101E500067657365747A7400434F4E534400446160
:101E600074656E2077657264656E20646972656B57
:101E70007420756562657274726167656E00434FA8
:101E80004E534900446174656E2077657264656ED7
:101E9000206765707566666572740000434F4E4238
:101EA0004500426C69747A2065696E676573636882
:101EB000616C74657400434F4E424100426C69741A
:101EC0007A206175736765736368616C746574000B
:101ED000434F4E4448004845582D44554D502076B8
:101EE000657277656E6465740000434F4E4442002E
:101EF00042696E616572646174656E617573676174
:101F000062650000434F4E4345005A757361657426
:101F10006C69636865204B6F6D6D656E7461726589
:101F20002065696E0000434F4E4341005A7573614E
:101F300065746C69636865204B6F6D6D656E746167
:101F4000726520617573000030303131303000002F
:101F500039310000460030303030414100004154FA
:101F60002B434D47533D00002B4300004665686CF2
:101F70006572206265696D2056657273656E646571
:0A1F80006E2E2052657472792E0057
:00000001FF
